:020000040000FA
:1000000000000000F5EF04F0800E016EFE0E81D8B6
:10001000010E7FD8750E0F6E300ECCD1016A018EA5
:100020001D6EFE0E76D81D5074D0066A800E326E9C
:1000300000D0166A176A186A196A099A75D8D30F18
:10004000D8B4098A2D0FC60FF9E20A0FF7E3126E32
:10005000116A106A0F6A0A0E0E6E31EC02F012502D
:100060000E24166E0F50176E000ED8B0010E172614
:100070001050186E000ED8B0010E18261150196ECF
:10008000000ED8B0010E1926060605E04DD8C60FA1
:1000900002E20A0FDCE209AA0BD0161E171E181E78
:1000A000191E162AD8B4172AD8B4182AD8B4192A6F
:1000B000165012000096065003E100860A0E066EE6
:1000C00021C011F020C010F01FC00FF01EC00EF0B4
:1000D000056A196A186A176A0A0E166E97D9052AF0
:1000E0000550065CF6E11650D8A4009600A602D092
:1000F000062C03D01650300F0CD8062EE1D7120074
:10010000A66AA68E0900F55003E011EC05F0FAD7B7
:10011000120001BE11EF05F001A202D001B08AD099
:1001200001B202D001B01FD032BEEE5012000088E2
:1001300000A8009800BA03D0008A34D828E20094BE
:1001400045D8C58643D8C95000B408D000B805D0FA
:10015000C59AC588C5B8FED700B819D8D890126E10
:100160001DD0008800A8009800BC05D0FE0B096EC9
:10017000008CD89013D000BE06D01A6E008E14D812
:10018000D8B005D01A5014D802E200A807D0C58410
:10019000C5B4FED7009C009E009A00941C80D8A095
:1001A0001C9012000DD801D005D8095000BA0109E1
:1001B000C96E0AD094869488C580C5B0FED7120057
:1001C000C582C5B2FED71200C7B4FED71268C550AB
:1001D0001F0B00D000D0D890D8B41200122EF7D741
:1001E000D88012000098008A008C008E008409D00C
:1001F000008800A8009800BA03D0008A39D82DE200
:100200000094080E136E44D81236132EFCD700B497
:1002100007D000B801D04ED849D845D800B81DD86D
:1002200047D8D890125020D0008A008C008E02D07F
:10023000008800A8009800BC05D0FE0B096E008C59
:10024000D89012D000BE05D01A6E008E11D805E2EB
:100250001A5012D802E200A807D02CD827D8009C48
:10026000009E009A009424D81C80D8A01C901200F4
:1002700017D8095000BA0109126E080E136E123613
:1002800017D801E217D812D80ED8132EF8D710D8E5
:100290000DD800D00000D89082B2D88004D81200C7
:1002A00007D804D807D88294949406D0948404D0B4
:1002B000948202D08B92949200D000D000D000D0D3
:1002C00012009482948400D000D000D000D08B948F
:1002D000949400D094841200EA6802C0E9FF071CDD
:1002E000E988E92AEC160E500F10D8B4120008D98C
:1002F00002C0E9FF0750EF1A000000D000D00E2A1C
:10030000D8B40F3EF9D7EF1A1200A96EA66AA680DC
:10031000A850A92A1200A86EA66AA684550EA76E38
:10032000AA0EA76EA682A6B2FED7A694A92A12008C
:10033000080E1A6EEA6803C0E9FF045009B4E5D854
:1003400009A4E5D8E26803C0E1FFEA6802C0E9FF5A
:10035000071CE988E92AEC161A50D8B4120009B033
:10036000C1D802C0E9FF0F320E32EF500710D8A0FB
:100370000718EF6E03D81A2EF6D712000450E71AAA
:10038000000000D000D000D000D000D000D000D0BD
:1003900000D000D0E71A1200136A126EFF0E122668
:1003A000132200D0D8A01200030E0F6EE60E02D862
:1003B000F5D70F6AFD0F0E6E01D00E06000000D0BB
:1003C000E86A0F5AFAE212000009D8B412001C6E53
:1003D0000EC0E9FF0FC0EAFF0F6A0E6A1CBE07D00D
:1003E000EE500E6E1CA21200EF500F6E120004D8D9
:1003F000EF14D8A40E2A1200010E1CB0E8441CB25F
:10040000E8441CB2E8441CB4E8381200266A276AA3
:10041000286A296A210E146E15D02636273628360A
:1004200029361650265C175027581850285819504E
:10043000295808E3296E1650265E1750275A18507F
:10044000285AD8800E360F3610361136142EE5D7BE
:1004500029C019F028C018F027C017F02650166ED2
:10046000120011C029F010C028F00FC027F00EC0F4
:1004700026F028501602F3CF10F0F4CF11F02750D9
:100480001702F3501026F450112226501802F35090
:100490001026F450112229501602F350112628502C
:1004A0001702F350112627501802F3501126265038
:1004B0001902F350112626501602F3CF0EF0F4CF96
:1004C0000FF027501602F3500F26F4501022000EA2
:1004D000112226501702F3500F26F4501022000E5E
:1004E00011221200126A136A04D00F320E32123631
:1004F0001336FF0FFAE213C00FF012500E6E120007
:100500000E1E0F1E0E4A0F2A1200EF1203D0FF0A12
:10051000EF1601D0FF0AE988E92AEC161200A66A54
:10052000A68E0900F55002E0EE6EFBD71200316A8C
:10053000306A7E0E2E6E800E2BAE000E2F6E01D80E
:1005400042D12E502A5C356E11E2356C2A502EC0F5
:100550002AF02E6E2B502FC02BF02F6E2C5030C057
:100560002CF0306E2D5031C02DF0316E1A0E3560EA
:1005700074D02E5272E0346A2B50386E2F18376EBA
:100580002B8E2F8E080E355E08E331C034F030C05C
:1005900031F02FC030F02F6AF5D7352607E0D8901C
:1005A0002F32303231323432352EF9D737AE33D0A4
:1005B00031502D5E30502C5A2F502B5A07E2D880E4
:1005C000000E2D562C562B56800E381A346C04E033
:1005D0002D06000E2C5A2B5A040E356E2B660DD0AC
:1005E0002CC02BF02DC02CF034C02DF0346A080E36
:1005F0002A5E29E3352EF2D726D02BBE08D0D8901C
:1006000034362D362C362B362A2EF7D71CD034AE66
:1006100022D0346A0FD031502D2630502C222F504A
:100620002B2206E32B322C322D3234322A4A0DD0C3
:1006300034AE11D02D3E0FD02C3E0DD02B3E0BD022
:10064000D8802D90EFD72A6A02D036822A682D6A88
:100650002C6A800E2B6E38AE2B9E2D5012002B5024
:10066000286E2F18376E2E5051E02A5252E02A5E23
:100670007F0E03E22A2603E24BD02A264CE22DC04D
:1006800026F02CC027F0288E2F8E180E386E2D6A7B
:100690002C6A2B6A0BD03150265C3050275811E35E
:1006A000276E286A3150265E0BD004E22F50285C5A
:1006B000F2E007E33150265E3050275A2F50285A77
:1006C000D8802D362C362B36263627362836382E2F
:1006D000ECD72BBE07D02A521BE037322A06382A25
:1006E0003736E3D707E23150265E3050275A2F5075
:1006F000285A17E32D3E15D02C3E13D02B3E11D097
:100700002B322C322D322A3E0CD005D0368604D026
:1007100036842A6A02D036822A682D6A2C6A800EB4
:100720002B6E37AE2B9E2D5012002B50286E2F189B
:10073000376E2A50D8A42E503AE02A267E0E03E3C4
:100740002A5E03E336D02A5E31E32DC026F02CC0AA
:1007500027F0288E2F8E2D6A2C6A2B6A180E386E81
:1007600028322732263206E331502D2630502C22F3
:100770002F502B222B322C322D32382EF1D72BBE7C
:1007800007D02D362C362B362A5210E02A06283474
:1007900016E32D3E14D02C3E12D02B3E10D0D88024
:1007A0002B322C322D322A3E0AD003D036842A6ACC
:1007B00002D036822A682D6A2C6A800E2B6E37AEE4
:1007C0002B9E2D5012002AC038F02B502DC02BF03C
:1007D0002D6E2D3638322D32366A2D36383602E3FC
:1007E0003684367E06E13680386A2D6A2C6A2B6A9A
:1007F0000BD0382803E0D8802D3206D0D8902D3287
:1008000002E1368201D0368636B604D036A20FD049
:1008100036B407D07F0E2D6EFF0E2C6E2B6E2A6E17
:1008200023D0800E2D6E01D02D6A000EF6D736B083
:10083000FBD72A6A9F0E3860EBD77E0E3864F4D758
:100840009E0E385C07E0D8902D322C322B322A32A3
:10085000382AF6D736A408D0D880000E2A562B5650
:100860002C562D562DAEE0D72A501200379E0AD0B6
:10087000379E2DAE07D0D880000E2A562B562C5608
:100880002D56378E960E386E2D5209E0080E3826FA
:100890002BC02AF02CC02BF02DC02CF011D02C52E4
:1008A0000FE1080E385E2B5007E1080E385E2A5023
:1008B00002E12D5010D02A6A2C6E2AC02BF02A6A31
:1008C0002CBE06D0D8902A362B362C363806F8D7D0
:1008D00037AE2C9E38502AC02DF02A6E2C502BC0DB
:1008E0002CF02B6E12002020202020202020202001
:1008F00020202020202000002020202020564B35C2
:10090000444A000020204469676974616C2056469F
:100910004F005573696E67204144393835302020C7
:10092000202000005573696E6720536935333531D7
:10093000612020200000433D43616E63656C2044CC
:100940003D536176652000002020202020202020BB
:1009500000003000000031000000320000003300D1
:1009600000003400000035000000360000003700B1
:10097000000038000000390000002F000000410096
:100980000000420000004300000044000000450059
:100990000000460000004700000048000000490039
:1009A00000004A0000004B0000004C0000004D0019
:1009B00000004E0000004F000000500000005100F9
:1009C00000005200000053000000540000005500D9
:1009D00000005600000057000000580000005900B9
:1009E00000005A00000030000000400E366E006A21
:1009F0000001280EC66E4F0EC86E800EC76E0F0E19
:100A0000C16E740ED36E400E9B6E926A040E936E8E
:100A1000946A03EE00F0ED6AE950EA10FCE1EF6A37
:100A20001FD1E8CF92F000B24CD04E0EB3EC00F0E4
:100A3000140EB3EC00F0340EB1EC00F04E0EB3EC3B
:100A400000F0140EB3EC00F0300EB1EC00F0140E18
:100A5000CCEC01F04E0EB3EC00F0140EB3EC00F051
:100A6000340EB1EC00F04E0EB3EC00F0140EB3EC0B
:100A700000F0300EB1EC00F0140ECCEC01F04E0E94
:100A8000B3EC00F0140EB3EC00F0240EB1EC00F067
:100A90004E0EB3EC00F0140EB3EC00F0200EB1ECEF
:100AA00000F0140ECCEC01F0280E936F70D80C0EF1
:100AB000936F6DD8060E936F6AD8800E936F67D8C8
:100AC000008292C093F0FE0E935D02E1976B12D00C
:100AD00097530DE1030E935D03E1080E986F06D066
:100AE000040E935D02E1986B01D051D801D005D876
:100AF000010E976F92C0E8FF1200F00E9315946FED
:100B00009339F00B956F050E9411966F98519613CB
:100B10004E0EB3EC00F0140EB3EC00F09651B1ECB5
:100B200000F0010E9411966F985196134E0EB3EC8F
:100B300000F0140EB3EC00F09651B1EC00F0010E91
:100B40009811966F4E0EB3EC00F0140EB3EC00F05B
:100B50009651B1EC00F0050E9511966F98519613D1
:100B60004E0EB3EC00F0140EB3EC00F09651B1EC65
:100B700000F0010E9511966F985196134E0EB3EC3E
:100B800000F0140EB3EC00F09651B1EF00F0F00E4F
:100B90009315946F9339F00B956F040E9411966F23
:100BA000985196134E0EB3EC00F0140EB3EC00F017
:100BB0009651B1EC00F098519411966F4E0EB3EC33
:100BC00000F0140EB3EC00F09651B1EC00F098C0B8
:100BD00096F04E0EB3EC00F0140EB3EC00F096510C
:100BE000B1EC00F0040E9511966F985196134E0ECD
:100BF000B3EC00F0140EB3EC00F09651B1EC00F041
:100C000098519511966F4E0EB3EC00F0140EB3ECA4
:100C100000F09651B1EF00F04E0EB3EC00F00A0E6A
:100C2000B3EC00F0300EB1EC00F04E0EB3EC00F07F
:100C3000000EB3EC00F0000EB1EC00F04E0EB3EC81
:100C400000F0010EB3EC00F00F0EB1EC00F04E0E10
:100C5000B3EC00F00D0EB3EC00F00F0EB1EF00F0AE
:100C60002AEF0BF004009B6B4E0EB3EC00F0150E58
:100C7000B3EC00F0E00EB1EC00F04F0EB3EC00F07E
:100C8000130EB3EC00F097EC00F09C6F9C1F9C39A6
:100C9000F00B9C6F9C390F0B9C6F9C5303E0010E73
:100CA0009B6F5AD04E0EB3EC00F0150EB3EC00F073
:100CB000D00EB1EC00F04F0EB3EC00F0130EB3EC1D
:100CC00000F097EC00F09C6F9C1F9C39F00B9C6F20
:100CD0009C390F0B9C6F9C5303E0020E9B6F3CD022
:100CE0004E0EB3EC00F0150EB3EC00F0B00EB1EC0C
:100CF00000F04F0EB3EC00F0130EB3EC00F097ECE5
:100D000000F09C6F9C1F9C39F00B9C6F9C390F0B63
:100D10009C6F9C5303E0030E9B6F1ED04E0EB3ECF2
:100D200000F0150EB3EC00F0700EB1EC00F04F0EB9
:100D3000B3EC00F0130EB3EC00F097EC00F09C6FF6
:100D40009C1F9C39F00B9C6F9C390F0B9C6F9C5324
:100D500003E0040E9B6F00D0320ECCEC01F0010ECC
:100D60009C53D8A4000E336E010E9B53D8A4000EE2
:100D7000331601E0996B000E9CB1010E336E010E2B
:100D80009B5D010ED8A4000E331602E0440E996F4D
:100D9000000E9CB3010E336E010E9B5D010ED8A4B4
:100DA000000E331602E0430E996F000E9CB5010E43
:100DB000336E010E9B5D010ED8A4000E331602E0C7
:100DC000420E996F000E9CB7010E336E010E9B5DB3
:100DD000010ED8A4000E331602E0410E996F000EEA
:100DE0009CB1010E336E020E9B5D010ED8A4000E65
:100DF000331602E0230E996F000E9CB3010E336E82
:100E0000020E9B5D010ED8A4000E331602E0390ECF
:100E1000996F000E9CB5010E336E020E9B5D010EA4
:100E2000D8A4000E331602E0360E996F000E9CB760
:100E3000010E336E020E9B5D010ED8A4000E331618
:100E400002E0330E996F000E9CB1010E336E030E5B
:100E50009B5D010ED8A4000E331602E0300E996F90
:100E6000000E9CB3010E336E030E9B5D010ED8A4E1
:100E7000000E331602E0380E996F000E9CB5010E7D
:100E8000336E030E9B5D010ED8A4000E331602E0F4
:100E9000350E996F000E9CB7010E336E030E9B5DED
:100EA000010ED8A4000E331602E0320E996F000E28
:100EB0009CB1010E336E040E9B5D010ED8A4000E92
:100EC000331602E02A0E996F000E9CB3010E336EAA
:100ED000040E9B5D010ED8A4000E331602E0370EFF
:100EE000996F000E9CB5010E336E040E9B5D010ED2
:100EF000D8A4000E331602E0340E996F000E9CB792
:100F0000010E336E040E9B5D010ED8A4000E331645
:100F100002E0310E996F120000EEA5F0080EF76E98
:100F2000E60EF66E8FEC02F0EF6A1200A5510A6E23
:100F3000300E0A5CBD6FA6510A6E300E0A5CBE6FA1
:100F4000BD510A0DF3CF1EF0F4CF1FF0BE511E2489
:100F5000BF6FBF51040D250814E3F86A520EF32445
:100F6000F66E090EF420F76E0900F5CF0EF00900B9
:100F7000F5CF0FF00900F5500900E4EC01F00EC0C8
:100F8000A1F000EEA5F0B651A1C0EBFF800E016EFE
:100F9000C00E0EEC00F000EEA5F0EE5003E011ECF8
:100FA00005F0FBD7B62BB76B12002AEF0BF050EC15
:100FB00001F0C00E14EC01F0CC5114EC01F0CD5155
:100FC00014EC01F02DEF01F050EC01F0C00E14EC28
:100FD00001F0CC5114EC01F050EC01F0C10E14EC16
:100FE00001F0F2EC00F0CD6F61EC01F02DEF01F0BB
:100FF000E3C02DF0E2C02CF0E1C02BF0E0C02AF0FD
:1010000036EC04F02DC0EBF02CC0EAF02BC0E9F078
:101010002AC0E8F0E7C02DF0E6C02CF0E5C02BF0C8
:10102000E4C02AF036EC04F02DC0EFF02CC0EEF056
:101030002BC0EDF02AC0ECF0EBC02DF0EAC02CF094
:10104000E9C02BF0E8C02AF0EFC031F0EEC030F07C
:10105000EDC02FF0ECC02EF02FEC03F02DC021F0EE
:101060002CC020F02BC01FF02AC01EF02D6A2C6A65
:101070002B6A860E2A6E21C031F020C030F01FC0CE
:101080002FF01EC02EF095EC03F0E3EC03F0C06FE0
:101090002BC0C1F02CC0C2F02DC0C3F0216A206A61
:1010A0001F6A800E1E6E2150DF03F3CF21F0205007
:1010B000DF03F3CF20F0F45021261F50DF03F3CFDE
:1010C0001FF0F4502026000E21221E50DF03F3CF24
:1010D0001EF0F4501F26000E20222122C0511E2691
:1010E000C1511F22C2512022C3512122000E1E5C79
:1010F000C06F020E1F58C16F000E2058C26F000E45
:101100002158C36FEBC021F0EAC020F0E9C01FF006
:10111000070EE825D8A002D03682FF0E1E6E21C031
:101120002DF020C02CF01FC02BF01EC02AF0EFC005
:1011300031F0EEC030F0EDC02FF0ECC02EF02FEC0F
:1011400003F0E3EC03F0C46F2BC0C5F02CC0C6F075
:101150002DC0C7F0216A206A1F6A800E1E6E21C052
:1011600011F020C010F01FC00FF01EC00EF0E3C041
:1011700019F0E2C018F0E1C017F0E0C016F031EC51
:1011800002F011C021F010C020F00FC01FF00EC0FF
:101190001EF0E7C025F0E6C024F0E5C023F0E4C06F
:1011A00022F025C011F024C010F023C00FF022C09F
:1011B0000EF0C7C019F0C6C018F0C5C017F0C4C003
:1011C00016F031EC02F011C025F010C024F00FC071
:1011D00023F00EC022F022501E5CC46F23501F5813
:1011E000C56F24502058C66F25502158C76FE7C0DF
:1011F000CBF0E6C0CAF0E5C0C9F0E4C0C8F0DEC07C
:10120000CCF0C9C0CDF0D3DEDE29CC6FC8C0CDF0A4
:10121000CEDE020EDE25CC6F030EC215CD6FC7DE0B
:10122000030EDE25CC6FC1C0CDF0C1DE040EDE257D
:10123000CC6FC0C0CDF0BBDE050EDE25CC6FCBC0C1
:1012400021F0CAC020F0C9C01FF0C8C01EF0000EB7
:101250001E141E6E000E1F141F6E0F0E2014206E23
:10126000000E2114216E0C0ED890213220321F3234
:101270001E32E82EF9D7256A246A236AC6C022F0F6
:101280000F0E22161E502210CD6F91DE060EDE25A7
:10129000CC6FC5C0CDF08BDE070EDE25CC6FC4C091
:1012A000CDF085D6116A106A0F6A800E0E6ED4C01A
:1012B00019F0D3C018F0D2C017F0D1C016F031EC3D
:1012C00002F011C021F010C020F00FC01FF00EC0BE
:1012D0001EF0000E1E5CC06F020E1F58C16F000E84
:1012E0002058C26F000E2158C36FC76BC66BC56B09
:1012F000C46BCB6BCA6BC96B010EC86FD0C0CCF08E
:10130000C9C0CDF054DED029CC6FC8C0CDF04FDEBF
:10131000020ED025CC6F030EC2151F6A1E6ED5516A
:101320001E10CD6F44DE030ED025CC6FC1C0CDF0B2
:101330003EDE040ED025CC6FC0C0CDF038DE050EE9
:10134000D025CC6FCBC021F0CAC020F0C9C01FF09F
:10135000C8C01EF0000E1E141E6E000E1F141F6E5D
:101360000F0E2014206E000E2114216E0C0ED8904A
:10137000213220321F321E32E82EF9D7256A246A24
:10138000236AC6C022F00F0E22161E502210CD6F07
:101390000EDE060ED025CC6FC5C0CDF008DE070EE0
:1013A000D025CC6FC4C0CDF002D617C1CEF000D886
:1013B000CEC0CCF0800ECD6FFADD2DEF01F017C15D
:1013C000CFF000D8CFC0CCF0CD6BF1DD2DEF01F028
:1013D000350E116EA40E106EE90E0F6E0E6AF3C07C
:1013E00019F0F2C018F0F1C017F0F0C016F006ECDA
:1013F00002F011C00CF110C00BF10FC00AF10EC0C9
:1014000009F10CC111F00BC110F00AC10FF009C1B4
:101410000EF0196A186A176A020E166E06EC02F0D0
:1014200029C00DF028C00CF027C00BF026C00AF030
:101430000A500B100C100D1006E001010907000EF8
:101440000A5B0B5B0C5B00010CC111F00BC110F0CF
:101450000AC10FF009C10EF0F3C019F0F2C018F084
:10146000F1C017F0F0C016F031EC02F011C0F7F047
:1014700010C0F6F00FC0F5F00EC0F4F0F7C011F098
:10148000F6C010F0F5C00FF0F4C00EF0010E196EAA
:101490007D0E186E760E176EBA0E166E06EC02F002
:1014A0000EC000F1F7C011F0F6C010F0F5C00FF05B
:1014B000F4C00EF0010E196E7D0E186E760E176ECA
:1014C000BA0E166E06EC02F029C0FBF028C0FAF046
:1014D00027C0F9F026C0F8F0FBC02DF0FAC02CF0C0
:1014E000F9C02BF0F8C02AF036EC04F02DC0FFF064
:1014F0002CC0FEF02BC0FDF02AC0FCF0F00E2D6ECB
:101500002C687F0E2B6E920E2A6EFFC031F0FEC04B
:1015100030F0FDC02FF0FCC02EF095EC03F02DC094
:10152000FFF02CC0FEF02BC0FDF02AC0FCF05D0ED9
:10153000316EBB0E306E3E0E2F6E970E2E6EFFC0BC
:101540002DF0FEC02CF0FDC02BF0FCC02AF02FECDB
:1015500003F02DC0FFF02CC0FEF02BC0FDF02AC020
:10156000FCF0FFC02DF0FEC02CF0FDC02BF0FCC045
:101570002AF0E3EC03F00101016F2BC002F12CC053
:1015800003F12DC004F1086B0F0E076F06690569A2
:1015900000018C51E8B82FD01A0EDE6F00C1DFF0C9
:1015A00004C1E3F003C1E2F002C1E1F001C1E0F0E7
:1015B00008C1E7F007C1E6F006C1E5F005C1E4F0B7
:1015C000F8EC07F02A0ED06F0CC1D4F00BC1D3F0A9
:1015D0000AC1D2F009C1D1F0D56B64DEB10ECC6F77
:1015E000A00ECD6FD7EC07F0100ECC6F4F0ECD6F65
:1015F000D7EC07F02ED0220EDE6F00C1DFF004C161
:10160000E3F003C1E2F002C1E1F001C1E0F008C182
:10161000E7F007C1E6F006C1E5F005C1E4F0F8EC3B
:1016200007F0320ED06F0CC1D4F00BC1D3F00AC159
:10163000D2F009C1D1F0D56B35DEB10ECC6FA00E62
:10164000CD6FD7EC07F0110ECC6F6C0ECD6FD7ECD1
:1016500007F01200640ECCEC01F00CEC06F004EC88
:1016600000F08C91320ECCEC01F004EC00F0800E16
:10167000016E0EEC00F0080EF76EF80EF66E80ECC0
:1016800000F0800E016EC00E0EEC00F0090EF76E39
:10169000040EF66E80EC00F0070E136ED00ECDEC4B
:1016A00001F0000E85EC01F0396E86EC01F03A6E27
:1016B00086EC01F03B6E86EC01F03C6E040E85EC8E
:1016C00001F03D6E86EC01F03E6E86EC01F03F6E5F
:1016D00086EC01F0406E080E85EC01F08B6F04EC97
:1016E00000F08B5325E1800E016E0EEC00F0090E28
:1016F000F76E120EF66E80EC00F0B9D881B409D006
:1017000040C090F03FC08FF03EC08EF03DC08DF0E5
:1017100008D03CC090F03BC08FF03AC08EF039C08A
:101720008DF04BD8030E136EE80ECDEC01F01DD0FA
:10173000800E016E0EEC00F0090EF76E240EF66EB0
:1017400080EC00F08C8381A48C93A6D8E86A81A4F5
:10175000010FD8B48C93D8A48C83B4D8030E136E25
:10176000E80ECDEC01F004EC00F0E0D0E86A81B4C2
:10177000010F8CB1010801E112008C8181A48C91D0
:101780008C3109E33CC090F03BC08FF03AC08EF042
:1017900039C08DF008D040C090F03FC08FF03EC0FF
:1017A0008EF03DC08DF0080E85EC01F08B6F8B53F1
:1017B00002E103D801D086D812000F6A0A0E0E6E1D
:1017C00092908080800E026E010E076E6CEC01F02C
:1017D0000A0ECCEC01F0819890C02DF08FC02CF057
:1017E0008EC02BF08DC02AF038EC04F05F0E316E05
:1017F000700E306E090E2F6E840E2E6E95EC03F077
:1018000097EC02F02DC04CF02CC04BF02BC04AF0EE
:101810002AC049F04AC04EF049C04DF04CC050F0CB
:101820004BC04FF0810E026E200E076E810E036ECC
:10183000080E046E096A4DC00EF098EC01F04EC01F
:101840000EF098EC01F04FC00EF098EC01F050C093
:101850000EF098EC01F00E6A98EC01F00F6A0A0E97
:101860000E6E810E026E100E076E6CEF01F0819805
:101870008196819A0F6A0A0E0E6E810E026E080E14
:10188000076E6CEC01F00F6A0A0E0E6E810E026E8E
:10189000100E076E6CEF01F03CC0F3F03BC0F2F0AD
:1018A0003AC0F1F039C0F0F08C99E8EC09F040C092
:1018B000F3F03FC0F2F03EC0F1F03DC0F0F08C8993
:1018C000E8EF09F0E86A8CB3010F81B4010801E187
:1018D000120081B414D050EC01F0C00E14EC01F0F1
:1018E000100E14EC01F0800E14EC01F02DEC01F060
:1018F000110ECC6F6C0ECD6FD7EC07F013D050ECFF
:1019000001F0C00E14EC01F0110E14EC01F0800E89
:1019100014EC01F02DEC01F0100ECC6F4F0ECD6FDA
:10192000D7EC07F08C8381A48C931200000E85EC19
:1019300001F0396E86EC01F03A6E86EC01F03B6EF8
:1019400086EC01F03C6E040E85EC01F03D6E86ECF9
:1019500001F03E6E86EC01F03F6E86EC01F0406EC9
:1019600081A403D02A0E916F02D0200E916F800EB9
:10197000016E0EEC00F0410E11EC05F0915111ECEE
:1019800005F03D0E11EC05F0200E11EC05F0520EA5
:1019900011EC05F0580E11EC05F0200E11EC05F0DD
:1019A000080E066E3CC021F03BC020F03AC01FF08C
:1019B00039C01EF05AEC00F0200E11EC05F081B495
:1019C00003D02A0E916F02D0200E916F800E016E0F
:1019D000C00E0EEC00F0420E11EC05F0915111EC2E
:1019E00005F03D0E11EC05F0200E11EC05F0540E43
:1019F00011EC05F0580E11EC05F0200E11EC05F07D
:101A0000080E066E40C021F03FC020F03EC01FF01F
:101A10003DC01EF05AEC00F0200E11EC05F0996B61
:101A200032EC06F0410E995D010ED8A4000E336E23
:101A3000420E995D010ED8A4000E33122A0E995D54
:101A4000010ED8A4000E3312230E995D010ED8A406
:101A5000000E3312D8B4FDD0410E995D03E1520E51
:101A6000896F02D0540E896F2A0E995D07E1080E26
:101A7000A96E000E8BEC01F0996B13D6230E995DC5
:101A800007E1080EA96E010E8BEC01F0996B09D6E7
:101A900004EC00F0800E016E0EEC00F0090EF76E03
:101AA000360EF66E80EC00F0410E995D15E1800E69
:101AB000016EC00E0EEC00F0520E11EC05F0580E47
:101AC00011EC05F0200E11EC05F03D0E11EC05F0C7
:101AD000200E11EC05F014D0800E016EC00E0EEC3D
:101AE00000F0540E11EC05F0580E11EC05F0200E2C
:101AF00011EC05F03D0E11EC05F0200E11EC05F097
:101B0000996B00EE80F0090EF76E480EF66E8FECC2
:101B100002F0EF6A8A6B32EC06F0300E995D02E259
:101B2000000E01D0010E336E3A0E995D010ED8B051
:101B3000000E331612E0080E8A5D0FE200EE80F010
:101B40008A5199C0EBFF995111EC05F08A2B010ED7
:101B5000136E2C0ECDEC01F0996B430E995D010EC6
:101B6000D8A4000E336E440E995D010ED8A4000E69
:101B70003312D1E0430E995DD8B4D8D6440E995DA6
:101B8000D8A467D0520E895D31E100EE80F015ECEB
:101B900000F0396E17C03AF018C03BF019C03CF0A5
:101BA000A96A39508BEC01F03A508BEC01F03B50B4
:101BB0008BEC01F03C508BEC01F081A409D03CC0CF
:101BC00090F03BC08FF03AC08EF039C08DF008D055
:101BD00040C090F03FC08FF03EC08EF03DC08DF011
:101BE0008B5302E1EADD01D057DE32D000EE80F007
:101BF00015EC00F03D6E17C03EF018C03FF019C064
:101C000040F0040EA96E3D508BEC01F03E508BEC81
:101C100001F03F508BEC01F040508BEC01F081A4BF
:101C200009D03CC090F03BC08FF03AC08EF039C074
:101C30008DF008D040C090F03FC08FF03EC08EF0D5
:101C40003DC08DF08B5302E1B8DD02D025DE3ADED7
:0A1C5000996BB6EC0BF06AD6FFD7D3
:020000040030CA
:0300010008191DBE
:020005008080F9
:060008000FC00FE00F40E5
:0200000400F00A
:0A000000224C170247823202000072
:00000001FF
